:1000000018308A0000280000FF00030E8301A100C1
:100010000A08A0008A010408A2007708A300780853
:10002000A4007908A5007A08A6007B08A70083131E
:1000300083128C308400001C1F280C184A288C3036
:100040008400801C25288C184D288C308400801E4C
:100050002B288C1A47288C308400001E31280C1A5B
:100060004428220884002308F7002408F800250803
:10007000F9002608FA002708FB0020088A00210E54
:100080008300FF0E7F0E09008A110A1207298A11C8
:100090000A1272298A110A122A2A8A110A12722E47
:1000A0000A108A100A1182070D340A342D342E34B6
:1000B0005434433400340A108A100A118207083479
:1000C000083402341F341F340034003400340A1062
:1000D0008A100A118207003445340A34413420342E
:1000E0005334493455340D34443452344A344E3444
:1000F000463443344B3454345A344C3457344834F3
:100100005934503451344F34423447340E344D3422
:10011000583456340F34003433340A342D342034F8
:100120000734383437340D342434343427342C3401
:1001300021343A34283435342234293432342334C7
:1001400036343034313439343F3426340E342E349E
:100150002F343B340F340A108A100A1182070534F9
:100160000D3411341434093400341A340B340F3480
:100170001234003400340C3403341C341D3416346F
:100180001734133401340A34103415340734063468
:1001900018340E341E340034003400341934003462
:1001A000033419340E34093401340D341A34143440
:1001B00006340B340F3412341C340C341834163417
:1001C00017340A340534103407341E3413341D3404
:1001D000153411340A108A100A11F13E03188A0AE4
:1001E00082000D340A340D340A34543454345934F2
:1001F0002D3443346F346E346E3465346334743468
:1002000020345634653472343A3420340034A9161C
:100210002908831687008312871E1529A912290829
:1002200083168700831287121B29A91229088316B7
:10023000870083128716E4080319242964080C1E1A
:100240001F299900E4014C29E30803194929620890
:10025000FA006108E10A0319E20A840083137A189C
:100260008317000883160317C400831203130C1AA4
:100270003C29831603173529990061085F3C031D4B
:100280004729E208031D4729E2014F30E100E3035B
:100290004C2983160C128312A9162908831687008D
:1002A0008312871E5A29A9122908831687008312F0
:1002B00087126029A91229088316870083128716DE
:1002C0000C128A110A1231288C1E64291808A80001
:1002D0001A08F800A81C6E291812181600008A11B6
:1002E0000A128729A9162908831687008312871EF8
:1002F0008029A9122908831687008312871286296C
:10030000A9122908831687008312871664297808A2
:10031000EA004E1CA729CE189D296908203C031825
:100320009D29A91029088316870083128714CE14EB
:100330001330E40083160C1683126A08113C031D67
:10034000A2294E116A08133C031DA7294E15EA087D
:100350000319C82969084F3C031CC6296608FA001E
:100360006508E50A0319E60A840083137A188317DF
:100370006A0880006508F03C031DC429E608031DD7
:10038000C429E601A030E500E90AC8290130AD0022
:10039000A9162908831687008312871ED629A91259
:1003A00029088316870083128712DC29A9122908DD
:1003B00083168700831287168C128A110A1231283D
:1003C000CC1CEC297C08083C031DEC290130831669
:1003D0000317C9068312031383160317C9080319E9
:1003E000F8297C0883120313B504FD29831603172B
:1003F0007C08FF3A83120313B50555308316860037
:100400008312350886000034CC1C122A03176108B9
:10041000083C03190D2A0313122A01308316C9065A
:100420008312031383160317C90803191E2A8312A4
:1004300061080313B504232A831603178312610886
:10044000FF3A0313B505553083168600831235082D
:1004500086000034291129088316870083120715A6
:10046000FD308F00C1308E006B08003A03193C2A22
:10047000013A03195D2C682E5530831686008312CD
:10048000060883160317C70083120313CC1C512AD6
:100490007608043C031D512A83160317C7098312EB
:1004A00003138316031747087605003A03195E2ADB
:1004B00083120313CE15612A8316031783120313C5
:1004C000CE110317B308031D6E2A0313CE196F2A2A
:1004D00001300317B30003107D0CB400031303179E
:1004E000B408031D472B7D08B4003308013A0313F9
:1004F0000319962A0B3A0319A12A013A0319AD2AC6
:10050000073A0319B92A013A0319C52A033A03190C
:10051000D12A013A0319E62A1F3A0319FB2A013AA4
:100520000319102B053A03191C2B442BCE199E2AB4
:100530000A300317B300B501A02A03130317B30150
:10054000462B031735100313CE1DA92A03173514A4
:1005500003130B300317B300462B0317B510031317
:10056000CE1DB52A0317B51403130C300317B300BF
:10057000462B031735110313CE1DC12A031735155A
:1005800003130D300317B300462B0317B5110313E4
:10059000CE1DCD2A0317B51503130E300317B30074
:1005A000462B031735120313CE1DD92A0317351610
:1005B00003137E08053C0318E22A0F300317B3002B
:1005C000E52A031314300317B300462B0317B512A3
:1005D0000313CE1DEE2A0317B51603137E08063C3F
:1005E0000318F72A10300317B300FA2A0313143044
:1005F0000317B300462B031735130313CE1D032B2C
:100600000317351703137E08073C03180C2B113012
:100610000317B3000F2B031314300317B300462B3B
:100620000317B5130313CE1D182B0317B5170313A8
:1006300014300317B300462B0317B3010313CE1D69
:10064000412B7508103C031D282B0330AD00412BB6
:100650007208FA007108F10A0319F20A8400831380
:100660007A1883170317350880007108303C031D82
:100670003F2B720B3F2B0130F2002030F100F50AC6
:1006800003130317462B03130317B301482BB403BB
:10069000B108031D2D2C7D08B1003008013A031369
:1006A0000319742B0B3A03197E2B013A03198C2B77
:1006B000073A03199A2B013A0319A82B033A031995
:1006C000B62B013A0319CD2B1F3A0319E42B013A3B
:1006D0000319FB2B053A0319092C013A0319182CAD
:1006E000433A0319262C2A2C83160317C9018312B7
:1006F0000313E0210A300317B0002C2C003003173D
:10070000321801308316C800C90083120313E02198
:100710000B300317B0002C2C00300317B218013037
:100720008316C800C90083120313E0210C3003179D
:10073000B0002C2C00300317321901308316C8008A
:10074000C90083120313E0210D300317B0002C2CD5
:1007500000300317B21901308316C800C900831294
:100760000313E0210E300317B0002C2C00300317C8
:10077000321A01308316C800C90083120313E02126
:100780007E08053C0318C92B0F300317B000CC2B93
:10079000031314300317B0002C2C00300317B21AC7
:1007A00001308316C800C90083120313E0217E08BC
:1007B000063C0318E02B10300317B000E32B0313A3
:1007C00014300317B0002C2C00300317321B0130FB
:1007D0008316C800C90083120313E0217E08073C7A
:1007E0000318F72B11300317B000FA2B0313153041
:1007F0000317B0002C2C00300317B21B01308316F6
:10080000C800C90083120313E02115300317B0009C
:100810002C2C013083160317C90083120313E02127
:1008200003107D0C7D070317B1005630B0002C2C4F
:10083000013083160317C90083120313E02103104C
:100840007D0D0317B1005630B0002C2C0317B001FA
:100850002C2C03130317B0012E2CB103B008031D79
:10086000592CF0080319532C03136F08FA006E0873
:10087000EE0A0319EF0A840083137A18831700081D
:100880000317B20003136E08203C031D4D2C6F0BA1
:100890004D2C0130EF001030EE00F0030317B101D2
:1008A0000130B000592C03134D1E5A2C1F30031772
:1008B000B20003130130EB00682E5530831686001A
:1008C0008312060883160317C70083120313CC1C78
:1008D000742C03176008043C0319702C0313742C48
:1008E0008316C7098312031383160317470883125D
:1008F0006005003A0319802C0313CE15822C0317D0
:100900000313CE110317E708031D8F2C0313CE1911
:10091000902C01300317E7000310620CE80003136A
:100920000317E808031D642D6208E8006708013A10
:1009300003130319B72C0B3A0319C22C013A0319FC
:10094000CE2C073A0319DA2C013A0319E62C033AA4
:100950000319F22C013A0319052D1F3A0319182D1A
:10096000013A03192B2D053A0319372D612DCE19A4
:10097000BF2C0A300317E700E901C12C031303174A
:10098000E701632D031769100313CE1DCA2C03174B
:10099000691403130B300317E700632D0317E910E5
:1009A0000313CE1DD62C0317E91403130C300317C1
:1009B000E700632D031769110313CE1DE22C031703
:1009C000691503130D300317E700632D0317E911B1
:1009D0000313CE1DEE2C0317E91503130E30031776
:1009E000E700632D031769120313CE1DFA2C0317BA
:1009F0006916031303176308053C0318022D0F3013
:100A0000E700042D1430E700632D0317E9120313E8
:100A1000CE1D0D2D0317E916031303176308063CBB
:100A20000318152D1030E700172D1430E700632D43
:100A3000031769130313CE1D202D03176917031322
:100A400003176308073C0318282D1130E7002A2DEF
:100A50001430E700632D0317E9130313CE1D332D64
:100A60000317E917031314300317E700632D031767
:100A7000E7010313CE1D5E2D03175F08103C031D15
:100A8000462D05300313AD005E2D03175C08FA00F8
:100A90005B08DB0A0319DC0A840083137A188317C6
:100AA000690880005B085B3C031D5C2D5C0B5C2DC2
:100AB0000130DC004B30DB00DF0A03130317632D2A
:100AC00003130317E701652DE803E508031D442E12
:100AD0006208E5006408013A03130319912D0B3AEB
:100AE00003199B2D013A0319A92D073A0319B72DB4
:100AF000013A0319C52D033A0319D32D013A0319FD
:100B0000E82D1F3A0319FD2D013A0319122E053A5B
:100B10000319202E013A03192F2E433A03193D2EB3
:100B2000412E83160317C9018312031304220A30CE
:100B30000317E400432E00300317661801308316B4
:100B4000C800C9008312031304220B300317E4000A
:100B5000432E00300317E61801308316C800C90081
:100B60008312031304220C300317E400432E0030D9
:100B70000317661901308316C800C90083120313D6
:100B800004220D300317E400432E00300317E6194A
:100B900001308316C800C9008312031304220E30EB
:100BA0000317E400432E00300317661A0130831642
:100BB000C800C90083120313042203176308053C0D
:100BC0000318E52D0F30E400E72D1430E400432E28
:100BD00000300317E61A01308316C800C9008312DB
:100BE0000313042203176308063C0318FA2D103080
:100BF000E400FC2D1430E400432E00300317661B84
:100C000001308316C800C90083120313042203179E
:100C10006308073C03180F2E1130E400112E153025
:100C2000E400432E00300317E61B01308316C80092
:100C3000C90083120313042215300317E400432E66
:100C4000013083160317C900831203130422031013
:100C50000317620C6207E5005630E400432E0130B2
:100C600083160317C900831203130422031003170A
:100C7000620DE5005630E400432E0317E401432ED5
:100C800003130317E401452EE503E408031D652E55
:100C9000CA080319652E4908FA004808C80A03194A
:100CA000C90A840083137A1883170008E6004808ED
:100CB000463C031D612E490B612E0130C9003630C0
:100CC000C800CA03E5010130E4000313EB01682EFC
:100CD0002911290883168700831207110C108A1125
:100CE0000A1231288316851183128515AA0B8A2EC4
:100CF0007D30AA00AB0A2B083B3C031D8A2EAB01BA
:100D0000AC0A2C08023C031D8A2EAC01F830B60553
:100D10003608850083168511831285118C108A117F
:100D20000A1231286308103C031D9B2EE3080319A7
:100D30009B2E6400962E6008FA005F08DF0A0319F4
:100D4000E00A840083137A18831783160317410877
:100D50008000831203135F085F3C031DB52EE0087B
:100D6000031DB52EE0014F30DF00E30A83160C1699
:100D700083120034831603174108F8014002031858
:100D8000C42E4008F700D02EF7010830C200C00D75
:100D9000F70D410877020318F700F80DC20BC72EB4
:100DA000831203130034F701F80183160317400878
:100DB00003104118F707F70CF80CC118F707F70CE8
:100DC000F80C4119F707F70CF80CC119F707F70CE5
:100DD000F80C411AF707F70CF80CC11AF707F70CD3
:100DE000F80C411BF707F70CF80CC11BF707F70CC1
:100DF000F80C831203130034831603173D08C00058
:100E00006430C10083120313BA26780883160317CF
:100E1000BE003E08C0006430C10083120313D32615
:100E2000780883160317BD02831203134E1A1F2F6F
:100E300083160317BE0803192A2F831203133030B9
:100E4000831603173E07C000C100831203139226C6
:100E5000831603173D08C0000A30C1008312031334
:100E6000BA26780883160317BF003F08C0000A306F
:100E7000C10083120313D326780883160317BD021B
:100E8000831203134E1A512F83160317BE0803193A
:100E90004C2F83120313512FBF0803195C2F8312A9
:100EA00003133030831603173F07C000C1008312BD
:100EB000031392268316031730303D07C000C1008C
:100EC0008312031392260034BC3084008317000879
:100ED00003197C2F0630F800BF30F7006400F70BD1
:100EE0006E2FF80B6C2F7A30F700F70B752F000080
:100EF00000006400800B6A2F003483160317BC01C6
:100F00003C0883120313502000380319932F8316D3
:100F10000317BC0AC100831203139226831603171A
:100F2000802F8312031383160317BB013A083B0279
:100F30000318AF2F2C30C100831203139226903078
:100F4000831603173B07840083170008BC00BD000D
:100F500083120313FC2683160317BB0A962F0D304A
:100F6000C1008312031392260A3083160317C100AF
:100F7000831203139226A91029088316870083126F
:100F80008714643083160317BC008312031364278D
:100F9000A91029088316870083128710003483164E
:100FA00003179001043091009201930101309400E5
:100FB00095010630BA00831203137D27003483168F
:100FC00003173A083C020318E72F3C08BA003B0815
:100FD0003A020318ED2F3B08BA003A08F8008312D2
:040FE00003130034C3
:1010000083160317B8013808073C031C3428B03096
:101010003807B90042303807840083130008BA004B
:1010200083128E018316390883128D0083163A08C5
:1010300083128C0083168C130C15831203130B0878
:10104000F7008B138316031755308D00AA308D00DF
:101050008C148C1829280C117708831203138B0425
:1010600083160317B80A032883128E01A0308D005F
:1010700003134A0803178C0083168C130C15831274
:1010800003130B08F7008B138316031755308D00DD
:10109000AA308D008C148C184B280C117708831201
:1010A00003138B0403178E01A1308D0003134B082B
:1010B00003178C0083168C130C15831203130B0873
:1010C000F7008B138316031755308D00AA308D005F
:1010D0008C148C1869280C117708831203138B0465
:1010E00003178E01A2308D0003134C0803178C00E8
:1010F00083168C130C15831203130B08F7008B1344
:101100008316031755308D00AA308D008C148C186F
:1011100087280C117708831203138B0403178E01A1
:10112000A3308D0003134D0803178C0083168C1316
:101130000C15831203130B08F7008B138316031788
:1011400055308D00AA308D008C148C18A5280C11F8
:101150007708831203138B040034831603173908AE
:101160003C3A831203130319C2287E3A0319C52897
:10117000093A0319C8282F3A0319CB280A3A031948
:10118000CE28D1285730F800D3284F30F800D32884
:101190004730F800D3283530F800D3282330F80042
:1011A000D3280030F80000340130831603173902C9
:1011B000FC3E0318ED28043E83120313F22801308D
:1011C000F800F1284030F800F1281030F800F1283C
:1011D0000430F800F128831603170030F80083125A
:1011E000031300340A108A100A118207DF28E2284C
:1011F000E528E8280130831603173902FC3E03185E
:101200001329043E8312031318290230F80017290A
:101210008030F80017292030F80017290830F8002E
:101220001729831603170030F800831203130034C4
:101230000A148A100A118207052908290B290E2988
:101240004C1C2529AA30B50027290830B500831683
:101250000317380883120313B4003408013A031942
:101260004729033A03194729013A03195229073A32
:1012700003195729013A03195729033A0319572922
:101280000C3A03196B29013A03196F2974293308A1
:1012900083160317B90083120313AD2078080317D0
:1012A000E2007829013033020317E2007829300880
:1012B00083160317B90083120313AD207808FD00CD
:1012C000330883160317B90083120313AD2078087F
:1012D0000317E20078290830B50003177829AA30EF
:1012E000B5000317782903130730AD00922A0317BE
:1012F0000313B701FF30B800B901BA01BB01BC014B
:10130000BD01BE01BF01C001C1012F088316031733
:10131000B90083120313D4207808F6002F0883162F
:101320000317B90083120313FA207808FC002E0873
:10133000FE00320883160317B90083120313D4206A
:1013400078080317E0000313320883160317B90067
:1013500083120313FA2078080317E10003133108FE
:101360000317E3007C080313B50403176108031394
:10137000B504CC18B51135088600B60136088500CD
:1013800003178E0190308D000313340803178C006F
:1013900083168C130C15831203130B08F7008B13A1
:1013A0008316031755308D00AA308D008C148C18CD
:1013B000D7290C117708831203138B0403178E01AE
:1013C00092308D0003132E0803178C0083168C13A4
:1013D0000C15831203130B08F7008B1383160317E6
:1013E00055308D00AA308D008C148C18F5290C1105
:1013F0007708831203138B0403178E0191308D003D
:1014000003132F0803178C0083168C130C158312FB
:1014100003130B08F7008B138316031755308D0049
:10142000AA308D008C148C18132A0C1177088312A3
:1014300003138B0403178E0193308D0003133008C0
:1014400003178C0083168C130C15831203130B08DF
:10145000F7008B138316031755308D00AA308D00CB
:101460008C148C18312A0C117708831203138B0407
:1014700003178E0195308D000313310803178C007C
:1014800083168C130C15831203130B08F7008B13B0
:101490008316031755308D00AA308D008C148C18DC
:1014A0004F2A0C117708831203138B0403178E0144
:1014B00094308D000313320803178C0083168C13AD
:1014C0000C15831203130B08F7008B1383160317F5
:1014D00055308D00AA308D008C148C186D2A0C119B
:1014E0007708831203138B0403178E0196308D0047
:1014F0000313330803178C0083168C130C15831207
:1015000003130B08F7008B138316031755308D0058
:10151000AA308D008C148C188B2A0C11770883123A
:1015200003138B04003483160317B7013708073CF5
:10153000031CAA2A423037078400831337088A1114
:10154000831203135B208A15F800800083160317AB
:10155000B70A962A483083120313CA00CB01CC0184
:10156000CD010020AE01AF01B001B101B201B30164
:101570000A3083160317B8008312031320210317C0
:101580008E0180308D0001308C0083168C130C1579
:10159000831203130B08F7008B13831603175530C0
:1015A0008D00AA308D008C148C18D42A0C11770869
:1015B000831203138B0403178E0181308D008C017D
:1015C00083168C130C15831203130B08F7008B136F
:1015D0008316031755308D00AA308D008C148C189B
:1015E000EF2A0C117708831203138B04FA30831649
:1015F0000317900091010230BA008A11831203137D
:101600007D278A15643083160317BC008A11831264
:10161000031364278A1500342914290883168700C8
:10162000831207182D2B1E3083160317BC008A1156
:101630008312031364278A15291429088316870047
:10164000831207182D2B291429088316870083126B
:10165000071C232B0130F8002F2B0030F8008A15CF
:101660000A16622983160317B2013208073C031CCD
:101670004F2B4230320784008313B0303207B5005D
:1016800083128E018316350883128D0083168C1306
:101690000C1483120C0880008316B20A352B8312B7
:1016A0008E01A0308D0083168C130C1483120C084D
:1016B0000313CA0003178E01A1308D0083168C130B
:1016C0000C1483120C080313CB0003178E01A230F5
:1016D0008D0083168C130C1483120C080313CC009A
:1016E00003178E01A3308D0083168C130C14831204
:1016F0000C080313CD008A150A166B2903178E01F7
:1017000090308D0083168C130C1483120C08031375
:10171000B40003178E0192308D0083168C130C14C5
:1017200083120C080313AE0003178E0191308D0055
:1017300083168C130C1483120C080313AF000317C9
:101740008E0193308D0083168C130C1483120C08B9
:101750000313B00003178E0195308D0083168C1390
:101760000C1483120C080313B10003178E0194307C
:101770008D0083168C130C1483120C080313B20013
:1017800003178E0196308D0083168C130C14831270
:101790000C080313B3008A150A166E293408013A9F
:1017A0000319E82B033A0319022C013A0319162CEA
:1017B000073A0319352C013A03194F2C033A031940
:1017C000692C0C3A03198F2C013A03198F2C9C2C8D
:1017D0000130831603179000023091008312031327
:1017E00032088316031792008312031333088316FB
:1017F000031793000430BA008A11831203137D2764
:101800008A159F2C02308316031790000130910037
:101810008312031332088316031792000330BA00B1
:101820008A11831203137D278A159F2C0330831698
:1018300003179000910083120313320883160317D5
:101840009200831203133308831603179300831245
:10185000031331088316031794000530BA008A1168
:10186000831203137D278A159F2C043083160317D8
:10187000900002309100831203133208831603177D
:101880009200831203133308831603179300043066
:10189000BA008A11831203137D278A159F2C053005
:1018A000831603179000023091008312031330084F
:1018B000831603179200831203133208831603174B
:1018C00093000430BA008A11831203137D278A150E
:1018D0009F2C06308316031790000430910083126A
:1018E00003132F0883160317920083120313300883
:1018F000831603179300831203133208831603170A
:1019000094008312031333088316031795000630DF
:10191000BA008A11831203137D278A159F2C34087D
:1019200083160317900091010230BA008A118312C6
:1019300003137D278A159F2C0630AD009F2C0034A1
:1019400083160317BA01380883126A02031DAC2CF0
:101950000130F800DD2CDD2C0130831638078312AE
:101960006A02031DDA2C8316B901013083126A0260
:10197000831639020318C42CA0303907840083175A
:101980000008BA07B90AB52C013083126A02A03EDA
:1019900084008317000883163A02031DD52C0130FA
:1019A000F8008312DD2CD92C83160030F800831246
:1019B000DD2CDD2C0030F800DD2C03130034831601
:1019C00003173708643C031DE82C6430F800F82C3A
:1019D00037084B3C031DEF2C4B30F800F82C370830
:1019E000423C031DF62C4230F800F82C3C30F80045
:1019F000831203130034F030831603179000013074
:101A00009100370892000330BA008A118312031341
:101A10007D278A150034831603173808BA00BB01E6
:101A20000130BC008A1183120313DF278A1578085E
:101A300083160317B8003708013A831203130319FA
:101A40002B2D033A0319302D013A0319352D073A8E
:101A500003193A2D412D023083160317B900532D77
:101A6000043083160317B900532D01308316031772
:101A7000B900532D203083160317B900532D83125C
:101A80000313F030831603179000013091000530E6
:101A900092000330BA008A11831203137D278A153E
:101AA000752D83160317B80803195D2D39088312A5
:101AB0000313B604622D831603173908FF3A831205
:101AC0000313B605360885001430831603179000FB
:101AD0000230910037089200380893000430BA00B1
:101AE0008A11831203137D278A1500348316031786
:101AF0003708013A831203130319882D033A031997
:101B00008D2D013A0319922D073A0319972D9E2D19
:101B1000023083160317B800A32D04308316031771
:101B2000B800A32D013083160317B800A32D203071
:101B300083160317B800A32D83120313FF30F80098
:101B4000B92D831603178312031336088316031760
:101B50003805003A0319B42D0130F800831203133D
:101B6000B92DB92D831603170030F8008312031323
:101B7000B92D00340230831603172107B700B800CF
:101B800083120313A024F8080319752F8316031773
:101B90002008003A831203130319F92D013A03199F
:101BA000072E153A0319132E3C3A0319452E013A14
:101BB0000319452E183A0319452E773A0319452E75
:101BC000013A0319452E0F3A0319452E013A03191C
:101BD000452E033A0319452E013A0319452E793A49
:101BE0000319F22E073A0319F22E6F3A0319202F28
:101BF000652F83160317A108031D062E8A11831271
:101C00000313CF278A157C2F831603176F2F831694
:101C10000317A108031D122E83120313CE237C2F5A
:101C2000831603176F2F83160317210B442E2208E8
:101C3000043C031C342E1430900002309100220822
:101C400092002208B70083120313762578088316C2
:101C5000031793000430BA008A11831203137D27FF
:101C60008A15412E83160317F03090000130910041
:101C7000053092000330BA008A11831203137D27C6
:101C80008A157C2F831603176F2F83160317A1085D
:101C9000031DF12E2008283A831203130319692E1D
:101CA000013A0319762E183A0319832E773A03194D
:101CB000902E013A03199D2E0F3A0319AA2E013ACC
:101CC0000319B72E033A0319C42E013A0319D12E72
:101CD000DE2E831603173410831203134C1C752E4B
:101CE00083160317341483120313DE2E831603178F
:101CF000341083120313CC1C822E83160317341462
:101D000083120313DE2E831603173410831203137A
:101D10004D1D8F2E83160317341483120313DE2EEA
:101D2000831603173410831203134D1C9C2E831645
:101D30000317341483120313DE2E83160317341093
:101D400083120313CD1CA92E831603173414831298
:101D50000313DE2E83160317341083120313CD1DD5
:101D6000B62E83160317341483120313DE2E831644
:101D700003173410831203134D1EC32E831603174B
:101D8000341483120313DE2E8316031734108312C8
:101D90000313CD1ED02E831603173414831203139E
:101DA000DE2E831603173410831203134D1FDD2E0E
:101DB00083160317341483120313DE2E83160317BE
:101DC000200890000130910092013418920A0330EB
:101DD000BA008A11831203137D278A157C2F83167C
:101DE00003176F2F83160317A108031D1F2F200849
:101DF000323A831203130319012F073A0319082FEC
:101E00000F2F4A08831603179200831203130F2F14
:101E10004B08831603179200831203130F2F8316A8
:101E2000031720089000013091000330BA008A1196
:101E3000831203137D278A157C2F831603176F2FB8
:101E400083160317A108031D622FB5013508073C4F
:101E5000031C542F02303507B60020085A3A83126B
:101E60000313031D502F9030831603173607F80015
:101E70000130FA000318FA0A7808B7007A08B800A7
:101E800042303507840083130008B9003708840006
:101E90008313381883173908800083120313502FD7
:101EA00083160317B50A262F2008900008309100EA
:101EB0000A30BA008A11831203137D278A157C2FFA
:101EC000831603176F2F8312031302308316031731
:101ED000B70083120313FB247C2F831603170330F0
:101EE000B70083120313FB247C2F033083160317E0
:101EF000B70083120313FB248A110A161D2DB901A2
:101F00008316031732080A3A831203130319982F12
:101F1000073A03199B2F2D3A03199E2F2E3A0319C6
:101F2000A12F013A0319A42F083A0319A72FAE2FA6
:101F30000230F800F22F0830F800F22F0430F800D9
:101F4000F22F1B30F800F22F1F30F800F22F203054
:101F500083160317B20083120313AE2F83160317E1
:101F60003208603C0318BB2F32087A3C031CBB2F9D
:101F70003208DF39BC2F3208B20032081F3C031888
:101F8000ED2F32085A3C031CED2F3208403C031C55
:101F9000D52F8312031338081B3C0319D22F1B3093
:101FA000B800B900DE2F8316031783120313380815
:101FB0001F3C0319DE2F1F30B800B90020308316F4
:101FC000031732028A1183120313AB208A15F8001B
:101FD000F800F22FF22F831603170030F800831257
:061FE0000313F22F003490
:102000000230831603172107B700B8000A128A1599
:1020100083120313A0240A168A11F8080319C02B8F
:10202000831603172008013A831203130319582853
:10203000033A03199528013A0319C528073A0319E9
:102040001129013A03195129033A031991290C3A2C
:102050000319FE29013A0319FE291F3A03191F2A01
:102060003C3A0319342A013A0319342A183A03195D
:10207000342A773A0319342A013A0319342A0F3AD9
:102080000319342A013A0319342A033A0319342A6A
:10209000013A0319342A793A0319EB2A073A03194A
:1020A000EB2A6F3A03193A2BA03A0319962BA82B67
:1020B000831603172108023C031D9428831203137F
:1020C000AE01AF01B0010530B1008316031722083D
:1020D000BA000130BB000430BC000A1283120313A3
:1020E000DF270A167808B200831603172308B70003
:1020F0000A128A1583120313DF240A168A1178083C
:10210000B300013083160317B8000A128A15831230
:10211000031320210A168A110A128A15CE230A16E1
:102120008A11CB2B83160317B62B83160317210BAB
:10213000C42883120313AE01AF01B0010830B1000F
:10214000831603172208BA000130BB000430BC001C
:102150000A1283120313DF270A167808B2006E30C2
:10216000B300023083160317B8000A128A158312CF
:10217000031320210A168A110A128A15CE230A1681
:102180008A11CB2B83160317B62B8316031721084E
:10219000033C031D102983120313AE01AF01B001EC
:1021A000831603172408BA000530BB000830BC00B2
:1021B0000A1283120313DF270A167808B100831668
:1021C00003172208BA000130BB000430BC000A1219
:1021D00083120313DF270A167808B2008316031749
:1021E0002308BA000430BB00FF30BC000A1283127F
:1021F0000313DF270A167808B3000330831603178A
:10220000B8000A128A158312031320210A168A11B4
:102210000A128A15CE230A168A11CB2B83160317AE
:10222000B62B831603172108023C031D50290530E5
:1022300083120313AE000430AF0083160317230884
:10224000B7000A128A1583120313DF240A168A11B3
:102250007808B0000530B100831603172208BA00D1
:102260000130BB000330BC000A1283120313DF27C6
:102270000A167808B2003008B3000430831603173A
:10228000B8000A128A158312031320210A168A1134
:102290000A128A15CE230A168A11CB2B831603172E
:1022A000B62B831603172108023C031D9029053025
:1022B00083120313AE000430AF0083160317220805
:1022C000B7000A128A1583120313DF240A168A1133
:1022D0007808B0000830B100831603172308BA004D
:1022E0000130BB000330BC000A1283120313DF2746
:1022F0000A167808B2006E30B30005308316031753
:10230000B8000A128A158312031320210A168A11B3
:102310000A128A15CE230A168A11CB2B83160317AD
:10232000B62B831603172108043C031DFD29053035
:1023300083120313AE00831603172208BA0001307C
:10234000BB000430BC000A1283120313DF270A16F5
:102350007808AF00831603172308B7000A128A15FE
:1023600083120313DF240A168A117808B00005309F
:10237000B100831603172408BA000130BB000430F3
:10238000BC000A1283120313DF270A167808B20072
:10239000831603172508B7000A128A158312031340
:1023A000DF240A168A117808B30032082F020319B5
:1023B000EF29330830020319EF290630831603177B
:1023C000B8000A128A158312031320210A168A11F3
:1023D0000A128A15CE230A168A11CB2BFB29043048
:1023E00083160317B7000A128A1583120313FB24FE
:1023F0000A168A11CB2B83160317B62B83160317E5
:10240000A108031D1E2A83120313AE01AF01B00100
:10241000B101B201B301831603172008B8000A12F4
:102420008A158312031320210A168A110A128A15AB
:10243000CE230A168A11CB2B83160317B62B8316CD
:1024400003172108023C031D332A2208B700230882
:10245000B8000A128A15831203130B250A168A1173
:10246000CB2B83160317B62B83160317210BEA2AEF
:10247000A20803193D2A34143E2A34102008283AB1
:102480008312031303195D2A013A03196A2A183AC1
:102490000319772A773A0319842A013A0319912AF2
:1024A0000F3A03199E2A013A0319AB2A033A03197A
:1024B000B82A013A0319C52AD22A4C1083160317E9
:1024C000341C672A831203134C14831603178312D8
:1024D0000313D22ACC1083160317341C742A8312D8
:1024E0000313CC148316031783120313D22A4D113E
:1024F00083160317341C812A831203134D15831688
:10250000031783120313D22A4D1083160317341CAA
:102510008E2A831203134D14831603178312031399
:10252000D22ACD1083160317341C9B2A831203135F
:10253000CD148316031783120313D22ACD118316E9
:102540000317341CA82A83120313CD15831603170F
:1025500083120313D22A4D1283160317341CB52A93
:10256000831203134D168316031783120313D22A03
:10257000CD1283160317341CC22A83120313CD16FF
:102580008316031783120313D22A4D1383160317DE
:10259000341CCF2A831203134D178316031783129B
:1025A0000313D22A0A128A1500200A168A118316EA
:1025B0000317200890000130910092013418920A0C
:1025C0000330BA000A12831203137D270A16CB2B9D
:1025D00083160317B62B83160317210B392B2008FC
:1025E000323A831203130319F92A073A03190F2BFE
:1025F000242B831603172208BA000A30BB00503080
:10260000BC000A1283120313DF270A167808CA00D7
:102610004A0883160317920083120313242B831690
:1026200003172208BA00BB010630BC000A1283124D
:102630000313DF270A167808CB004B08831603170D
:10264000920083120313242B0A128A1500200A1603
:102650008A1183160317200890000130910003307F
:10266000BA000A12831203137D270A16CB2B831696
:102670000317B62B831603172108083C031D952B5F
:10268000B5013508073C031C7E2B02303507B60028
:1026900020085A3A83120313031D7A2B4230831603
:1026A00003173507B700B8010318B80AA03036077A
:1026B000840083170008B900370884008313381892
:1026C00083173908800090303607B7000130B80012
:1026D0000318B80A42303507840083130008B90094
:1026E0003708840083133818831739088000831251
:1026F00003137A2B83160317B50A412B0A128A1586
:102700008312031300200A168A1183160317200868
:102710009000083091000A30BA000A1283120313A5
:102720007D270A16CB2B83160317B62B83160317A8
:10273000A108031DA52B0A128A15831203139322E5
:102740000A168A11CB2B83160317B62B8312031399
:10275000023083160317B7000A128A158312031377
:10276000FB240A168A11CB2B831603170330B700FC
:102770000A128A1583120313FB240A168A11CB2B23
:10278000033083160317B7000A128A158312031346
:10279000FB240A168A118A110A161D2D83160317A7
:1027A000B401831203134E1CE62BCE1CE62BE90862
:1027B000031DE62BA91029088316870083128710B2
:1027C000CE101130E40083160C168312E9080319A9
:1027D000042C6808FA006708E70A0319E80A84006D
:1027E00083137A188317000883160317B400831223
:1027F00003136708F03C031D032CE808031D032C9A
:10280000E801A030E700E903831603173408F80055
:102810007808B20083120313CE1E272C83160317E9
:10282000B20803191C2C3208C1000A1283120313C8
:1028300092260A168316031732080D3C031D292C15
:102840000A30C1000A128312031392260A16831655
:1028500003173208003A831203130319392C2F3A55
:1028600003193C2C223A0319472C073A0319472C29
:102870005A2C0030F8001F2D01300317EB002F30C9
:10288000EC0083163208F800831203131F2D031780
:102890006B08023C031D532CEA0A0930EB000313BA
:1028A0005A2C5A2C0317EB0183163208F8008312B6
:1028B00003131F2D03176B08013A03130319672C29
:1028C000033A0319842C0B3A0319F52CF92C8316BF
:1028D000031732082C3C031D7B2C02308312EB00C3
:1028E000EA018316A0013208F800831203131F2D9A
:1028F000842C8316031732088312EC0683163208E1
:10290000F800831203131F2D8316031732082C3C83
:10291000031DA02C8312EA0A6A08103C031D922CA6
:10292000EB01022DA0306A07840083178001831613
:102930003208F800831203131F2DF52C831603179A
:1029400032082F3C0318D92C3208393C031CD92CEF
:10295000A03083126A078316B4000130B500031853
:10296000B50AA03083126A07840083170008831613
:10297000B6000A30C0003608C1000A1283120313E1
:10298000D3260A16780883160317B70030303202B0
:102990003707B800340884008313351883173808C4
:1029A00080003208F800831203131F2DF52C8316C4
:1029B00003173208583C031DED2CA03083126A0720
:1029C00084008317FF30800083163208F8008312DA
:1029D00003131F2DF52C831603178312EB018316A7
:1029E0003208F800831203131F2D0317EB01022D89
:1029F00003130317EB0183163208F8008312031345
:102A00001F2D03176C08023A031303190B2D053A07
:102A100003190C2D112D00280A128A15BA2D0A1639
:102A20008A11013083160317B7000A128A15831220
:102A30000313FB240A168A111D2DDA30F800003426
:102A400003174A08103C031D2A2D04300313AD0060
:102A5000442D03174708FA004608C60A0319C70A97
:102A6000840083137A188317831636088000831234
:102A70004608463C031D422D470B422D0130C7003E
:102A80003630C600CA0A031300347D30AA00AB01F9
:102A9000AC01831603173308003A8312031303199A
:102AA000552D013A0319222E7F2E83160317B208E3
:102AB00003191F2E831203134B08013A0319642DC7
:102AC000023A0319802D812D320883160317B700AF
:102AD0000A128A158312031376250A168A11F8083A
:102AE000031D7F2D320883160317B7000130B8008D
:102AF0000A128A15831203130B250A168A11822DD6
:102B0000822D822D4D1DBE2D831603173208083AE3
:102B1000831203130319962D133A0319982D043ABF
:102B20000319982D1D3A0319982D992DBB019B2D42
:102B30009B2DBB0A9B2D4A083B02031CBE2DBB01EB
:102B400083160317B4013408073C031CBC2D423024
:102B500034078400831380080319BA2D42303407E8
:102B6000840083130008B500B600831203132025E8
:102B700083160317B40AA32D8312031338081B3CD2
:102B8000031DFB2D4D1CD72D831603173208043C63
:102B90000319CD2D83120313D72D1F308312031376
:102BA000B80083160317B600831203132025CD1C2B
:102BB000EC2D831603173208083C0319E22D83120B
:102BC0000313EC2D1F3083120313B8008316031771
:102BD000B600831203132025CD1DFA2D831603178B
:102BE00032081B3C0319F72D83120313FA2D882E8C
:102BF00083120313092ECD1D092E831603173208E5
:102C00001F3C0319062E83120313092E882E8312EC
:102C100003138316031732081B3C031D152E1B30AC
:102C200083120313B8008316031732081F3C031DD9
:102C30001F2E1F3083120313B8008316031783124D
:102C400003137F2E83160317B20803197C2E8312F9
:102C500003134B08013A031D492E3208831603174C
:102C6000B7000A128A158312031376250A168A11F1
:102C7000F808031D482E320883160317B7000130E9
:102C8000B8000A128A15831203130B250A168A113B
:102C9000492E4D1D7E2E8316031732080D3C031D51
:102CA000572E83120313BB015A2E83160317831268
:102CB0000313BB0A4A083B02031C7E2EBB010D30E6
:102CC00083160317B6008312031320250A308316D8
:102CD0000317B60083120313202583160317B401CC
:102CE0003408033C031C7C2EB601831203132025F9
:102CF00083160317B40A702E831203137F2E8316D4
:102D000003173208B6008312031320258316031716
:102D100083120313003483160317B2018312DF08F2
:102D20000319AB2E5E08FA005D08DD0A0319DE0AFE
:102D3000840083137A18831700088316B200831265
:102D40005D085B3C031DAA2E5E0BAA2E0130DE003F
:102D50004B30DD00DF0383163208F80083120313C3
:102D600000348316031732081F3A83120313031922
:102D7000BD2E043A0319C62ED02EB701CD1AC52E8A
:102D800083160317B20183120313D02E2030B7002D
:102D9000CD1ACF2E83160317B20183120313D02E40
:102DA00037088316031732070A12831203136720AA
:102DB0000A16F800F800003483160317B201F5086C
:102DC0000319F92E7408FA007308F30A0319F40AB8
:102DD000840083137A1883170008B2007308303C0C
:102DE000031DF82E740BF82E0130F4002030F30090
:102DF000F5033208F8008312031300347008103C06
:102E0000031D052F0230AD00202F6D08FA006C085D
:102E1000EC0A0319ED0A840083137A1883178316CA
:102E2000031732088000831203136C08203C031D33
:102E30001F2F6D0B1F2F0130ED001030EC00F00A3A
:102E40000034F930831603179000013091003208E6
:102E500092000330BA000A12831203137D270A1668
:062E60008A150A16812B01
:10300000840183131F30830583161F149F141F151B
:103010009F1120309900263098009030831298003C
:10302000A801FF30A9007D30AA00AB01AC01AD01C1
:10303000AE01AF01B001B101B201B301B401B501FC
:10304000B601B701B801B901BA01BB01BC01BD01AC
:10305000BE01BF01C001C101C201C301C401C5015C
:10306000C601C701C801C901CA01CB01CC01CD010C
:103070004E10CE104E11E0014F30DF00E201E100B2
:10308000E301E401E601A030E500E801E700E90121
:10309000EA01EB01CE110130ED001030EC000130FF
:1030A000EF001030EE00F0010130F2002030F100AE
:1030B0000130F4002030F300F5010430F600083050
:1030C000FC005730FD000530FE000317B001B101D0
:1030D000B201B301B401B5010130C7003630C600FA
:1030E0000130C9003630C800CA010130DC004B3065
:1030F000DB000130DE004B30DD00DF010130E0009D
:103100000230E1005730E2000530E300E401E50160
:10311000E601E701E801E9018316900191019201BE
:1031200093019401950196019701980199019A01E3
:103130009B019C019D019E019F01831203134E126E
:103140000317EA01EB010313CE1283161F149F1419
:103150001F159F110030850083128501553083169D
:103160008600AA3083128600993083168700831266
:10317000A900403087004E14CE124E120830F700DE
:10318000F71DCB28073081018130840083130008AC
:10319000C0390F3880006400813084000008C039D5
:1031A0007704800083168C16C03083128B04113094
:1031B0000C1ED828990083160317B20132080A1290
:1031C0008A1183120313EA200A168A15003803199C
:1031D000F92883160317B20AC1000A128A11831252
:1031E000031392260A168A1583160317DE28831204
:1031F0000313013083160317BD000A128A118312CC
:103200000313FC260A168A152E3083160317C100F5
:103210000A128A118312031392260A168A1583163C
:103220000317BD010A128A1183120313FC260A1622
:103230008A150D3083160317C1000A128A118312F2
:10324000031392260A168A150A3083160317C10043
:103250000A128A118312031392260A168A150A1279
:103260008A11CF270A168A15643083160317BC000B
:103270000A128A118312031364270A168A15031788
:103280008E0180308D0083168C130C1483120C0871
:10329000013C031950290A12031393220A1603173B
:1032A0008E0181308D0083168C130C1483120C0850
:1032B00003195F290A12031393220A1603170A122D
:1032C00003130C2B0A16F808031969290A12932212
:1032D0000A160A12322B0A160A127E2B0A16340814
:1032E00083160317B8000A128312031320210A164B
:1032F0000A12CE230A164830F80006389200FA3037
:10330000831692008312910183168C1485308312E8
:103310009000FD308F00C1308E0083160C14831294
:103320003408013A0319A429033A0319FC29013A84
:103330000319FC29073A03194F2A013A0319822A73
:10334000033A0319DC2A6C2B0317CA08031DDA2978
:103350008A110313CE238A15780883160317B10048
:10336000B1080319D9293108B2000A1283120313D4
:103370007F270A16780883160317B00083120313F9
:10338000B9080319CD29390883160317B200B30110
:103390008A118312031345258A15831603173008F3
:1033A000B200B3018A118312031345258A158316CF
:1033B000031783128A1103138B268A157808831644
:1033C0000317B000B0080319FB293008B2008A11B6
:1033D00083120313B1268A15780883160317B000E9
:1033E0003008C1000A128A118312031392260A16AA
:1033F0008A1583160317742B0317CA08031D382A6E
:103400008A110313CE238A15780883160317B10097
:10341000B1080319372A3108DA3C031D1A2A0D3086
:10342000B6008A118312031320258A150A308316E9
:103430000317B100831203133408023C031D2C2A26
:10344000831603173108B2000130B3008A118312CA
:10345000031345258A15352A831603173108B6004C
:103460008A118312031320258A15831603178312EA
:103470008A1103138B268A15780883160317B00068
:10348000B00803194E2A3008C1000A128A118312AB
:10349000031392260A168A1583160317742B8A11B2
:1034A000CE238A15780883160317B1008A11831278
:1034B0000313DC268A15780883160317B000B008BA
:1034C00003196C2A3008B200B3018A118312031366
:1034D00045258A15831603178A11831203138B2639
:1034E0008A15780883160317B000B0080319812ADB
:1034F0003008B2008A1183120313FE268A15831640
:103500000317742B8A11CE238A15780883160317A4
:10351000B1008A1183120313DC268A1578088316FA
:103520000317B000B0080319AB2A3008B2008A11A3
:1035300083120313B1268A15780883160317B00087
:103540003008B2000130B3008A11831203134525FD
:103550008A15831603178A11831203138B268A1583
:10356000780883160317B000B0080319DB2A300867
:10357000B2000A12831203137F270A1678088316F3
:103580000317B00083120313B9080319D02A3908AE
:1035900083160317B2008A1183120313FE268A15BD
:1035A000831603173008B2008A1183120313FE2614
:1035B0008A1583160317742B300833020318262B41
:1035C0008A11DC268A15780883160317B000B00824
:1035D0000319F52A3008C1000A128A118312031355
:1035E00092260A168A15831603178312CA08031D2A
:1035F0000F2B8A110313CE238A157808831603171D
:10360000B100B10803190E2B3108B200B3018A11C1
:103610008312031345258A158316031783128A1113
:1036200003138B268A15780883160317B000B00899
:103630000319232B3008B2008A1183120313FE26CC
:103640008A1583160317692B831203138A118B269D
:103650008A15780883160317B000B00803193B2BAE
:103660003008C1000A128A118312031392260A1627
:103670008A1583160317F008031D532B8A11831232
:103680000313CE238A15780883160317B100B108F7
:103690000319532B3108B2008A1183120313FE263B
:1036A0008A15831603178A1183120313DC268A15E1
:1036B000780883160317B000B0080319692B300887
:1036C000B200B3018A118312031345258A158316AC
:1036D0000317742B831203138A11CE238A157808DB
:1036E00083160317B100742B83120313AD0803195B
:1036F000832B2D0883160317B2008A11831203133C
:0E370000212F8A15AD01640083168F29630006
:02400E00723FFF
:02FFFE00760883
:0840000000000B0002000200A9
:00000001FF
